:1000000003C003C003C003C003C003C003C003C0D8
:1000800039C35BC35AC359C358C357C356C355C3B7
:1000900054C353C352C351C350C34FC34EC317C0FD
:1000A000197A4005930B0902120001010080320900
:1000B000040000000000000012011001FF00000811
:1000C000D0165307040200000001040309041124A0
:1000D0001FBECFE5D2E0CDBFDEBF20E0A0E6B0E09E
:1000E00001C01D92AC38B207E1F7BFC1A82FB92FEC
:1000F00080E090E041E050EA609530E009C02D9149
:1001000082279795879510F084279527305EC8F34E
:100110006F5FA8F30895EADF8D939D930895CF93C1
:10012000CFB7CF93C395B39BE9F7B39B0BC0B39BFA
:1001300009C0B39B07C0B39B05C0B39B03C0B39B6F
:1001400001C0D9C00F92DF93C0916E00DD27CA585D
:10015000DF4F012EB39B03C0DF910F90E6CF2F93AB
:100160000F931F934F932FEF4F6F06B303FB20F9AD
:100170005F933F9350E03BE065C016B301265029E2
:1001800053FDC89556B3012703FB25F92F7306B31A
:10019000B1F05027102713FB26F906B22230F0F0F9
:1001A00000C016B3012703FB27F90126502906B228
:1001B0002430E8F54F77206816B30000F6CF5027BB
:1001C0004F7D206206B2102F000000C006B300264B
:1001D0005029102713FB26F906B2E2CF4F7B06B356
:1001E000206400C0DACF01265029187106B269F1E7
:1001F0004E7F2160012F16B328C0002650294D7F65
:1002000006B22260102F29C0012650294B7F06B26A
:100210002460012F2DC016B301265029477F286086
:10022000000006B22EC04F7E06B3206130C04227C8
:1002300006B3499300265029102706B24FEF13FB4F
:1002400020F9297F16B379F2187159F10126502946
:1002500006B2012703FB21F9237F06B371F20026C2
:1002600050293150D0F006B2102713FB22F9277E17
:1002700016B351F201265029012703FB06B223F9D8
:100280002F7C49F2000006B3102713FB24F9002647
:10029000502906B22F7939F270CF10E21ABF002729
:1002A0001DC03B503195C31BD04010E21ABF0881DE
:1002B000033C29F10B3419F120916C001981110FC5
:1002C0001213EDCF093651F10D3211F0013E39F71D
:1002D000CAE01AB715FD02C0CA95D9F70093740099
:1002E0003F915F914F911F910F912F91DF910F904F
:1002F000CAB7C5FD17CFCF91CFBFCF910895209139
:100300007400222369F3109172001123F1F4343048
:10031000F2F03093720020936D0019C000917200CA
:1003200001309CF40AE530916F0034FD11C0009358
:100330006F00C1E6D0E010C0052710E000C021C06A
:10034000052710E0C89508BB14C03AE501C032ED9E
:10035000032EC0E0D0E032E017B31861C39A08B3AF
:1003600017BB58E120E84FEF20FF052708BB279572
:1003700017951C3F28F700004552B0F720FF0527CE
:10038000279508BB17951C3FB8F629913A9561F758
:10039000077E10917300110F08BBC250D04011F0BE
:1003A00010936C0010E21ABF086017B3177E402F3D
:1003B000477E54E05A95F1F708BB17BB48BB90CF76
:1003C0002FEFB0E8A0E04AE0B1BF000081EE9CE072
:1003D000B399FECFB39BFECF0197B399FDCF97FFA3
:1003E00003C0BA1B819501C0BA0FA69539F4A0E4E9
:1003F00028F4281710F031B7282FA1E0415021F739
:1004000031BF00000895F201309741F02AE742160B
:1004100029E1520629F481B790E002C08FEB9CECF1
:1004200021E00C0120935700E8951124CF0102969A
:100430002C01089514BE88E181BD87E081BDBB9A7F
:100440002FE28BE19FE0215080409040E1F700C017
:100450000000BB988AE580936F008FEF8093600067
:10046000AC9A8BB780628BBF0895B898C09A8CE124
:1004700090E10197F1F700C00000EAE7F9E1E491AB
:10048000EF3F11F0E1BF0000B09B06C0EDE7F9E1DE
:10049000E491EF3F09F02BC1CDDF712C312C412CC1
:1004A000512CCCE7D5E114E686B3887109F014E647
:1004B000115029F41092730010926C0081DF0AB67B
:1004C00005FE04C02CDE80E28ABF02C0219761F7DE
:1004D000A895832D823069F4E0E8F9E1E054F10950
:1004E00083E080935700E8953097C1F7412C512C59
:1004F00012C0803459F4F2013297E03899E1F907DB
:1005000050F485E080935700E89505C0843019F4D5
:10051000CD2B11F4E9C0312C80917200835087FDFE
:100520009AC090916D009D3209F093C0883009F017
:1005300090C083EC809361008AE580936F00809186
:100540007700807690917800882381F1712C911149
:1005500008C082E899E1909371008093700086E072
:100560006DC0913069F441145104F1F080917B0029
:10057000807C482E50907C0081E187BFE89514C0B4
:10058000933081F48091790090917A003CDF8091E2
:100590007B0090917C0037DF842D8F7329F490E4E9
:1005A000392E4CC09F73392E80E048C0809179006D
:1005B00010926A00911106C010926B002AE630E09A
:1005C00082E038C0953019F48093730025C09630CE
:1005D000E9F490917A00913019F48AE999E104C024
:1005E000923041F488E899E1909371008093700013
:1005F00082E124C09330C1F68111D6CF8CEA99E113
:10060000909371008093700084E018C0983079F066
:10061000993031F4809375002AE630E080E00AC01A
:1006200081E09A3009F080E02AE630E003C025E757
:1006300030E081E0309371002093700090917E0053
:10064000911105C090917D00981708F4892F80932F
:1006500060001092720080916F0084FF2FC0809123
:1006600060008F3F59F1C82F893008F0C8E08C1B1B
:10067000809360009091610088E8892780936100F1
:10068000CC2381F0E0917000F0917100A2E6B0E01F
:100690008C2F94919D9331968150D9F7F0937100EE
:1006A000E09370006C2F82E690E035DDCC5FCC30BB
:1006B00019F08FEF80936000C0936F00C301019623
:1006C0003C01803B944029F4EDE7F9E1E491EF3FF0
:1006D00059F40AB605FEE5CE8DE1B39B8DE181505C
:1006E000E1F780E28ABFDDCEA5DE1BBE15BAC09859
:1006F000D4CCFFCF0000000000000000000000008C
:1007000000000000000000000000000000000000E9
:100710000000000011241FBECFE5D2E0DEBFCDBF38
:1007200010E0A0E6B0E0ECE9F9E002C005900D921F
:10073000A236B107D9F710D12FC1A2CC807C20E01E
:1007400030E0FC01E20FF31F45915491F901EE7F77
:10075000E60FF71F518340832E5F3F4F2034310552
:1007600081F70895FC01E07C93E090935700E895B1
:1007700007B600FCFDCF0895CF93DF939B01205C6B
:100780003F4FDB01FC01E61BF70BEA0FFB1FCD918E
:10079000DD9141E00E0140935700E8951124A21726
:1007A000B30781F725E0FC0120935700E89507B6D1
:1007B00000FCFDCFDF91CF910895CF93DF93CDB7AC
:1007C000DEB7C054D1090FB6F894DEBF0FBECDBF5F
:1007D000BE016F5F7F4F80E090E0B0DF8FEF9FEF53
:1007E0009A83898380E090E0BDDFBE016F5F7F4F19
:1007F00080E090E0C1DFC05CDF4F0FB6F894DEBF51
:100800000FBECDBFDF91CF9108950F931F93CF936C
:10081000DF93CDB7DEB7C054D1090FB6F894DEBF71
:100820000FBECDBF00E010E0003886E0180709F4E5
:1008300040C020E030E0F901E00FF11FE256FF4F29
:10084000C9019595879546E0E43FF40768F0880F65
:10085000991FE1E0F0E0EC0FFD1FE80FF91F8FEFAB
:100860009FEF918380830CC045915491880F991F0D
:10087000E1E0F0E0EC0FFD1FE80FF91F518340832A
:100880002E5F3F4F20343105B1F68091600090918A
:100890006100800F911F66DF809160009091610080
:1008A000BE016F5F7F4F800F911F66DF005C1F4F9F
:1008B000BBCFC05CDF4F0FB6F894DEBF0FBECDBF1D
:1008C000DF91CF911F910F9108950F931F93CF93B5
:1008D000DF93CDB7DEB7C054D1090FB6F894DEBFB1
:1008E0000FBECDBF80916000909161009695879575
:1008F00081509044FE0131969E012F5B3F4F8F0146
:1009000081939193E217F307D9F780E090E02ADF13
:10091000B80180E090E030DFC05CDF4F0FB6F894A4
:10092000DEBF0FBECDBFDF91CF911F910F91089514
:1009300087B3836087BBC1982AEF8DE190E1FC010A
:100940003197F1F7C19A0197F1F7C1982150A9F7B2
:100950000895E0E0F0E0099488B318BA87B38FEF08
:1009600087BB8AEF90E0EDE1F0E13197F1F7019775
:10097000D1F787B317BA8AEF90E0EDE1F0E1319754
:10098000F1F70197D1F7F89418DF3FDF9EDFD0DF52
:0C099000E0DF80E090E00895F894FFCFD5
:02099C008019C0
:040000030000008079
:00000001FF
